:100000000C941E060C9412280C943F280C9446065F
:100010000C9446060C9446060C9446060C94460630
:100020000C9446060C9446060C9422130C94460637
:100030000C9446060C9446060C9446060C94460610
:100040000C946C280C9446060C945A2C0C949D2C01
:100050000C9446060C9446060C9446060C944606F0
:100060000C9446060C9446068618E818C718CA1859
:10007000CD18D018D318D618D918E818E2181A1ABB
:100080001C1A1C1A1A1A1C1A1C1A1C1A1C1A1C1AC2
:100090001C1A1C1A1C1A1C1A1C1A1C1A1C1A1C1AB0
:1000A000A0191C1A1C1A1C1A1C1A1C1A11191C1A29
:1000B0001C1A1C1A1C1A1C1A1C1A1C1A1C1A1C1A90
:1000C0001C1A1C1A1C1A1C1A1C1A1C1AAC19AC1962
:1000D000AC19AC19AC19AC19AC19AC19AC191C1A87
:1000E0001C1A1C1A1C1A1C1A1C1A1119AB19AB1950
:1000F000AB19AB191C1AB919BF19C519CB19D119EC
:10010000D719DD19E319ED19F719011A0B1A52194C
:1001100014191C1A1C1A1C1A1C1AA0191C1A1C1AB5
:100120001C1A1C1A1C1A1C1A1C1A1C1AAA19AA1905
:10013000AA19AA191C1AB919BF19C519CB19D119AD
:10014000D719DD19E319ED19F719011A0B1A52190C
:1001500014191C1A1C1A1C1A1C1AA0194F1A4F1A0F
:100160004F1A4F1A4F1A4F1A4F1A4F1A4F1A4F1A47
:100170004F1A4F1A4F1A661B661B661B661B661BBF
:10018000661B941A9E1AA81AB21A101B1A1B291B56
:100190003A1BC21CD71CE31CEC1CFB1C201D291D98
:1001A000721D3B1D85208B2091209820A620C82001
:1001B000E620456E746572206D656E752E2E2E00DC
:1001C000546F67676C6564206D6963726F50504D42
:1001D00000546F67676C656420696E76657274653C
:1001E000642050504D2100546F67676C6564205443
:1001F00058206D7574696E672100546F67676C6570
:10020000642074656C656D65747279210050726F3D
:10021000746F636F6C206572726F72207769746897
:100220002052580054696D656F7574207768656E4B
:1002300020636F6E6E656374696E6720746F205201
:100240005800507265737320616E79206B65792058
:10025000746F2063616E63656C00436F6E6E6563DF
:1002600074696E6720746F2052582C20706F776508
:100270007220757020746865205258202877697440
:10028000682062696E6420706C7567206966206EF4
:100290006F74207573696E6720616C776179732064
:1002A00062696E642900546F67676C656420276912
:1002B0006D6D656469617465206F75747075742700
:1002C00000546F67676C65642027736C61766520E6
:1002D0006D6F64652700546F67676C6564202761E4
:1002E0006C776179732062696E642700546F676769
:1002F0006C65642050504D206368616E6E656C20A3
:100300006C696D69740053657420525353492069B8
:100310006E6A656374696F6E206368616E6E656C8A
:100320002028303D3D64697361626C652900536526
:10033000742050504D206D696E696D756D20737914
:100340006E630053657420626561636F6E20696E31
:1003500074657276616C0053657420626561636FC9
:100360006E2064656C617900536574206265616319
:100370006F6E206672657175656E637920696E2097
:10038000487A3A20303D64697361626C652C205074
:10039000783D504D52206368616E6E656C20782CFC
:1003A0002046783D465253206368616E6E656C202E
:1003B00078005365742050574D2073746F7020641B
:1003C000656C61792028302064697361626C6564B2
:1003D0002C20312D323535203D3D20302E317320FB
:1003E0002D2035306D696E29005365742050504DB5
:1003F0002073746F702064656C61792028302064EC
:10040000697361626C65642C20312D323535203D75
:100410003D20302E3173202D2035306D696E29003E
:10042000536574206661696C736166652064656CF0
:1004300061792028302064697361626C65642C20C6
:10044000312D323535203D3D20302E3173202D2089
:1004500035306D696E29002A2A2A2A2A2A2A2A2A50
:100460002A2A2A2A2A2A2A2A2A2A2A2A2A2A2A2AEC
:100470002A2A2A2A0052582041636B6564202D20C5
:1004800072657665727420737563636573736675E0
:100490006C21002A2A2A2A2A2A2A2A2A2A2A2A2AAD
:1004A0002A2A2A2A2A2A2A2A2A2A2A2A2A2A2A2AAC
:1004B000002A2A2A2A2A2A2A2A2A2A2A2A2A2A2AC6
:1004C0002A2A2A2A2A2A2A2A2A2A2A2A2A2A00528E
:1004D000582041636B6564202D20757064617465DC
:1004E000207375636365737366756C21002A2A2A0D
:1004F0002A2A2A2A2A2A2A2A2A2A2A2A2A2A2A2A5C
:100500002A2A2A2A2A2A2A2A2A2A0056616C696457
:100510002063686F69636573206172653A205B319F
:100520005D2D5B31365D20286368616E6E656C20E1
:10053000312D31362900536574206F7574707574D0
:1005400020666F7220706F727420005B585D2061AE
:10055000626F7274206368616E67657320616E6498
:10056000206578697420525820636F6E6669670051
:100570005B535D20736176652073657474696E6783
:100580007320746F205258005B525D20726576654F
:1005900072742052582073657474696E6773207486
:1005A0006F2064656661756C747300557365206EA9
:1005B000756D62657273205B312D445D20746F2010
:1005C0006564697420706F727473205B452D515D92
:1005D00020666F722073657474696E677300202DD6
:1005E00020726563656976657220636F6E66696700
:1005F000757261746F722C20727820737720000AF4
:100600000A6F70656E4C52536E67200053657420FC
:1006100073657269616C2062617564726174653AB8
:10062000200056616C69642063686F696365733A82
:100630002031202D20342B34202F2032202D203823
:10064000202F2033202D20382B34202F2034202D14
:10065000203132202F2035202D2031322B34202FF5
:100660002036202D20313600536574204368616E9A
:100670006E656C20636F6E6669673A20005365741F
:100680002044617461726174652028302D32293AEA
:10069000200053657420486F70206368616E6E653A
:1006A0006C7320286D61782032342C207365706162
:1006B000726174656420627920636F6D6D61732966
:1006C0002076616C69642076616C75657320312DCC
:1006D0003235353A2000536574206368616E6E656B
:1006E0006C2073706163696E6720287831306B48C5
:1006F0007A293A200053657420524620706F77653E
:10070000722028302D37293A200053657420524634
:10071000206D6167696320286865782920652E67E8
:100720002E20307844454144463030443A2000532E
:1007300065742062617365206672657175656E63AC
:10074000792028696E20487A293A20005B5A5D207A
:10075000656E746572207265636569766572206383
:100760006F6E66696775726174696F6E2075746902
:100770006C79005B465D20646973706C61792061FF
:10078000637475616C206672657175656E63696509
:10079000732075736564005B525D2063616C6375E3
:1007A0006C6174652072616E646F6D206B65792079
:1007B000616E6420686F70206C697374005B495DC2
:1007C000207265696E697469616C697A6520736508
:1007D0007474696E677320746F20736B65746368DB
:1007E0002064656661756C7473005B585D2072658A
:1007F00076657274206368616E67657320616E64EC
:100800002065786974206D656E75005B535D20739B
:100810006176652073657474696E677320746F20E8
:10082000454550524F4D20616E64206578697420B3
:100830006D656E7500557365206E756D62657273BA
:10084000205B302D395D20746F20656469742070E1
:100850006172616D657465727300202D2053797328
:1008600074656D20636F6E66696775726174696F18
:100870006E000A0A6F70656E4C52536E672000510D
:1008800029204F7574707574206265666F726520DB
:100890006C696E6B20283D465329203A2000502970
:1008A00020536C617665206D6F64652028657870D3
:1008B0006572696D656E74616C293A20004F29205C
:1008C00054696D65642042494E44206174207374FC
:1008D000617274757020203A20004E292050504DCE
:1008E000206F7574707574206C696D69746564200F
:1008F000202020203A200044495341424C454400E6
:100900004D292050504D205253534920746F20637D
:1009100068616E6E656C202020203A20004C2920F2
:1009200050504D206D696E696D756D2073796E63E1
:10093000202875732920203A200044495341424C15
:100940004544004B29204661696C736166652062ED
:100950006561636F6E20696E74762E2028312D32AA
:10096000353573293A20004A29204661696C736144
:10097000666520626561636F6E2064656C617920D5
:1009800028302D323535203D3E20313073202D204A
:100990003135306D696E293A200049292046616958
:1009A0006C7361666520626561636F6E206672714B
:1009B0002E203A200048292050574D2073746F7024
:1009C0002064656C6179202020202020203A2000BE
:1009D00047292050504D2073746F702064656C61FE
:1009E00079202020202020203A200046292046611E
:1009F000696C736166652064656C617920202020D4
:100A00002020203A200050574D206368616E6E65AB
:100A10006C200066756E6374696F6E3A2000292041
:100A2000706F72742000506F776572546F776572C3
:100A300000445446205548462033322D62697420C4
:100A400031306368004F70656E4C52536E67525878
:100A5000206D696E6920342F36636800466C7974A6
:100A6000726F6E2F4F72616E6765525820554846FF
:100A70002038636800525820747970653A20004429
:100A8000697361626C656400487A00203D3D200016
:100A900043616C63756C61746564207061636B6540
:100AA0007420696E74657276616C3A200042292068
:100AB0004D6963726F202868616C66292050504D23
:100AC000202020203A00412920496E766572746505
:100AD000642050504D20696E20202020203A0030A4
:100AE00029204D7574652062757A7A657220286DAB
:100AF0006F73746C79293A003929205365726961E2
:100B00006C2062617564726174653A00736D617224
:100B100074506F7274004672536B79005472616E38
:100B200073706172656E740044697361626C6564B0
:100B30000038292054656C656D657472793A2020FF
:100B40002020202020003729204368616E6E656CCC
:100B500020636F6E6669673A202000362920446161
:100B60007461726174652028302D32293A2020206A
:100B700000352920486F70206368616E6E656C7364
:100B80003A2020202020003429204368616E6E65C1
:100B90006C2073706163696E673A202000332920EE
:100BA000524620706F7765722028302D37293A2001
:100BB0002020003229205246206D616769633A2067
:100BC0002020202020202020003129204261736530
:100BD000206672657175656E63793A202020000089
:100BE00000000700020100000304060000000000EE
:100BF00000000001020408102040800102040810D7
:100C00002001020408102004040404040404040263
:100C10000202020202030303030303000000002395
:100C2000002600290000000000250028002B0000FD
:100C3000000000240027002A00008B2D11241FBE75
:100C4000CFEFD8E0DEBFCDBF13E0A0E0B1E0E4E23B
:100C5000F1E602C005900D92A83CB107D9F716E065
:100C6000A8ECB3E001C01D92AE38B107E1F71CE07B
:100C7000CCE3DCE004C02297FE010E94942ECA332C
:100C8000D107C9F70E94C72D0C9490300C94000036
:100C900080917305813019F482E08093730580910F
:100CA0007305833019F484E0809373050895A89543
:100CB0000895DC01ED91FC910190F081E02D099502
:100CC00008952091740530917505382748E0C901D1
:100CD000880F991F37FF06C09C0151E2252750E17C
:100CE000352701C09C01415091F730937505209341
:100CF0007405089588E38093760580E092ECA1E086
:100D0000B0E08093770590937805A0937905B09330
:100D10007A0587E08093830580EC9AECA9E8B6E336
:100D200080937B0590937C05A0937D05B0937E0511
:100D300085E0809384058DEE9EEFADEABEED809355
:100D40007F0590938005A0938105B0938205E5E827
:100D5000F5E080E090E0863028F4DC01AE54BC4F32
:100D60002C9101C020E0219301968831910599F7DB
:100D700082E080939D058AE080939E05089580EC33
:100D800097EFAAEBB7E38093BB059093BC05A093C4
:100D9000BD05B093BE0580E090E0A0E0B0E5809393
:100DA000BF059093C005A093C105B093C205E3ECC5
:100DB000F5E080E081938F5F8031E1F70895A0E056
:100DC000B0E0E5EEF6E00C945D2ED82F0E94C2282C
:100DD0006115710581059105C9F30E94002F1092DC
:100DE0007F05109280051092810510928205C4E063
:100DF000812C912C54018A94C0907F05D09080055D
:100E0000E0908105F0908205FE2CED2CDC2CCC24AA
:100E10000E94FB2EA50194010E943C2E6C0D7D1DAD
:100E20008E1D9F1D60937F057093800580938105C3
:100E300090938205C15001F7DD2309F450C005E805
:100E400015E0E801A12CB12C62E3C62ED12CE12CD7
:100E5000F12C8881882309F442C0B39419F40E94CC
:100E60007A063DC00E94FB2EA70196010E943C2EEF
:100E7000E1E0E60FA5E8B5E08A2F801B8A1520F493
:100E80008D918E13F9CFE9CF2091840530E0A0E158
:100E9000B7E20E94D42D9B01AC01AE2FB0E00E94BE
:100EA000E32D40907B0550907C0560907D0570900F
:100EB0007E05640D751D861D971D4090BB055090E5
:100EC000BC056090BD057090BE05461657066806C5
:100ED000790618F2E993A39488E1A812BACFCDB7A6
:100EE000DEB7E0E10C94792E8436910520F4BC0144
:100EF00080E090E017C09C018E3B910528F42A55B4
:100F00003109AAE0B0E00CC0823D910528F4245BD1
:100F10003109A4E6B0E004C02D5C3109A8E5B2E0D7
:100F20000E94D42DA4E6B0E09B01AC010E94E32D09
:100F3000089590E08C599F4F0E947407089561E0D6
:100F400086E00E946F2960E086E00E94A82982E086
:100F50008093B00085E08093B10061E083E00E945F
:100F60006F2960E083E00E94A8290895CF93DF9362
:100F7000EC010097E9F061E086E00E94A8299E015B
:100F800040E050E068E478EE81E090E00E943C2E82
:100F90002F3F31054105510529F020F02FEF30E0BA
:100FA00040E050E02093B3008091B000806107C022
:100FB00060E086E00E94A8298091B0008F7E809337
:100FC000B000DF91CF91089560E08EE00E946F291C
:100FD00061E08FE00E946F2961E080E10E946F294B
:100FE00060E082E00E946F2961E084E00E946F2946
:100FF000089542E050E068E476E080E00E94F22745
:101000000895E3E0F0E089E080935700E491E67012
:1010100081E0E63009F080E00895CF93DF93C82F98
:101020000E940108882381F0DFB781E08093720578
:10103000F8940E94570688E180936000C093600096
:10104000C1110E945706DFBFDF91CF9108958F92A3
:101050009F92AF92BF92CF92DF92EF92FF92CF9387
:10106000FC01C0A5EC2FE770F0E0E658FC4FA08132
:10107000B0E0C7FF03C024E130E002C02FE030E061
:10108000FC0197A183E1989FF0011124E25CFE4FDF
:1010900080809180A280B380A20FB31F20E43FE143
:1010A0004DE750E00E94EE2DA50194010E941A2EFA
:1010B0008C2F887149F469017A01E0EDCE0EE7E0EA
:1010C000DE1EE11CF11C1BC0C7FF05C060E47AE80E
:1010D0008CE29EE004C060E07EEE8AEB9BE069015A
:1010E0007A01F8EBCF0EFBE0DF1EE11CF11CA5013D
:1010F00094010E941A2EC20ED31EE41EF51EC701D3
:10110000B60169517C4F8F4F9F4F28EE33E040E08E
:1011100050E00E941A2EA8EEB3E00E94E32DCF917A
:10112000FF90EF90DF90CF90BF90AF909F908F9007
:1011300008958F3F910551F048F0811522E0920704
:1011400038F08115934030F482E0089580E00895EE
:1011500081E0089583E00895A0E0B0E0E2EBF8E0DC
:101160000C94662EEB018A01B82FB695A0E0288179
:101170003981F80120832A813B8121832C813D81A3
:1011800022832E813F812383688179814A815B811B
:101190002C813D81EE81FF819F2F9295990F990FB0
:1011A000907C272F2370922B252F2370220F220F44
:1011B000922B232F23702295207F922BF80194836A
:1011C0000B5F1F4F2896AF5FBA1788F680FF24C0C9
:1011D000888199810E949908D82E8A819B810E94DA
:1011E0009908E82E8C819D810E949908F82E8E81A5
:1011F0009F810E949908F0E4DF9EA001112490E1F4
:10120000E99E90011124242B282BE4E0FE9EB001DE
:101210001124262BF8012083CDB7DEB7E7E00C942C
:10122000822E803223E0920708F1883E23E0920765
:1012300040F48F519340E4E096958795EA95E1F765
:101240000895803D27E0920718F48C5D934008953F
:10125000883928E0920768F4885C974074E0969596
:1012600087957A95E1F78D509C4F089580E090E046
:1012700008958FEF93E008958C30910540F4A4E039
:10128000880F991FAA95E1F7885D9C4F0895843FC8
:1012900023E0920718F484529C4F0895811524E0AE
:1012A000920740F48657934FF4E0880F991FFA9500
:1012B000E1F7089580E998E008959C013695279517
:1012C00025753575821B930B9C012373337396959B
:1012D00087959695879583739373820F931F9C01CF
:1012E00054E0369527955A95E1F7280F391F2F704E
:1012F0003F7041E051E0249FC001259F900D349F35
:10130000900D1124892F08954298882319F0000028
:10131000419A02C0000041980000429A00000895DE
:10132000429A000086B14298000081700895CF93E0
:10133000DF93D82F5C9A42985C98C8E08D2F807814
:101340000E948409DD0FC150C9F74298DF91CF9107
:1013500008958F770E9497090895CF93DF93D82F30
:10136000C8E08D2F80780E948409DD0FC150C9F735
:101370004298DF91CF910895CF93DF934298C8E0D0
:1013800080E0D82FDD0F0E9490098D0FC150C9F762
:10139000DF91CF9108950E94A9090E94BC095C9A2F
:1013A0000895A1E0B0E0E7EDF9E00C946B2E8068C1
:1013B00069830E9497096981862F0E94AD095C9A12
:1013C0002196E2E00C94872ECF93C0917F05C82729
:1013D000E82FF0E0EA58FA4F678589E70E94D109C3
:1013E0006C2F8DE30E94D1096C2F82E40E94D109F9
:1013F000CF91089586E20E94CB090895CF93DF93A1
:10140000EC016C818CE10E94D1096D818DE10E941B
:10141000D1096E818EE10E94D1096F8180E20E9424
:10142000D109688581E20E94D109698582E20E9422
:10143000D1096A8583E20E94D1096B8584E20E940A
:10144000D1096C8585E20E94D1096D858AE20E94EE
:10145000D1096E858EE60E94D1096F858FE60E94C4
:10146000D109688980E70E94D109698981E70E94D2
:10147000D1096A8982E70E94D109DF91CF9108954D
:10148000CF92DF92EF92FF92CF93DF936B017C01BB
:10149000C11488E3D8068CE9E8068CE1F80628F543
:1014A000C701B60120E836E948E950E00E941A2E4B
:1014B000E901689760E879E687E69FEF0E94F62DDC
:1014C0006C0D7D1D8E1D9F1DF2E0660F771F881F1E
:1014D000991FFA95D1F721E732E040E050E00E94F1
:1014E0001A2EF22EE32E80E421C0C701B60120E0BF
:1014F0003DE241E351E00E941A2EE901689760E065
:1015000073ED8EEC9EEF0E94F62D6C0D7D1D8E1DF1
:101510009F1D660F771F881F991F21E732E040E06B
:1015200050E00E941A2EF22EE32E80E66C2F6F718F
:10153000680F85E70E94D1096E2D86E70E94D109C8
:101540006F2D87E70E94D109DF91CF91FF90EF9037
:10155000DF90CF900895682F8DE60E94D1090895FD
:101560008F929F92AF92BF92CF92DF92EF92FF92B3
:10157000CF93DF93D82F83E00E94CB09809371052E
:1015800084E00E94CB098093700560E086E00E94B1
:10159000D10961E087E00E94D1096FE789E00E94EC
:1015A000D10965E08AE00E94D10962E18BE00E94E6
:1015B000D10965E18CE00E94D1096DEF8DE00E94B8
:1015C000D10960E08EE00E94D109DD2319F08BE2A1
:1015D00091E008C020919D0533E1239FC0011124B3
:1015E000825C9E4F0E94FE096CE880E30E94D10954
:1015F0006FE082E30E94D10962E483E30E94D10993
:1016000080919E0587FF02C064E101C06AE084E327
:101610000E94D1096AE285E30E94D1096DE286E366
:101620000E94D10964ED87E30E94D10960E088E35C
:101630000E94D10960E089E30E94D109D11109C05B
:10164000C0907F05D0908005E0908105F0908205E4
:1016500007C0C5E9CC2EC1ECDC2EED2CCEEDFC2E66
:10166000CAE38F2C9924AA24BB24682D8C2F0E94B6
:10167000D109682D85E08C0F0E94D109FE2CED2C3C
:10168000DC2CCC24CF5FCE3361F76FEF83E40E9474
:10169000D1096FEF84E40E94D1096FEF85E40E94C5
:1016A000D1096FEF86E40E94D109DD2311F066E0D5
:1016B00002C0609183058DE60E94D10960E089E750
:1016C0000E94D109609184058AE70E94D10960E0F7
:1016D00083E70E94D10960E084E70E94D109D1111B
:1016E00009C060917B0570917C0580917D0590918A
:1016F0007E0504C060EC7AEC89E896E30E94400A1B
:10170000DF91CF91FF90EF90DF90CF90BF90AF909F
:101710009F908F90089561E087E00E94D10964E274
:101720008EE70E94D10963E088E00E94D10960E061
:1017300088E00E94D10965E087E00E94D10962E05B
:1017400085E00E94D10983E00E94CB098093710556
:1017500084E00E94CB0980937005089583E00E9485
:10176000CB098093710584E00E94CB0980937005BA
:1017700061E087E00E94D1096AE070E080E090E0DB
:101780000E94E5280E948B0B00000895CF92DF9203
:10179000FF920F931F93CF93DF931F92CDB7DEB7C6
:1017A000082F162F8EE399830E94D109F02EC02EA8
:1017B0009981D92E8C2D8F19811738F4F6016191FA
:1017C0006F018FE70E94D109F5CF64E085E00E94A8
:1017D000D10983E00E94CB098093710584E00E94C7
:1017E000CB09809370050E94C22860936C057093AA
:1017F0006D0580936E0590936F0569E087E00E9408
:10180000D10981E0809373050F90DF91CF911F91F3
:101810000F91FF90DF90CF9008950F931F930E9438
:10182000C60B80917305813099F40E94C228009103
:101830006C0510916D0520916E0530916F05601B50
:10184000710B820B930B603A76488140910548F307
:1018500080917305813031F46EE971E082EE95E09C
:101860000E94AE2A1F910F9108950F931F938091AC
:101870007305823021F41092730581E020C08091BD
:1018800073058130D9F40E94C22800916C05109133
:101890006D0520916E0530916F05601B710B820BF9
:1018A000930B613A76488140910540F061E087E012
:1018B0000E94D1091092730582E001C080E01F915F
:1018C0000F910895CF93DF93EC014AE050E06D2F24
:1018D00070E082EE95E00E947C2B6EE282EE95E055
:1018E0000E94802ABE0184E0769567958A95E1F78B
:1018F0006F7077274AE050E082EE95E00E947C2BE3
:101900006EE282EE95E00E94802ABE016F7077271A
:101910004AE050E082EE95E00E947C2BDF91CF916F
:101920000895D82FC0E0CD1790F4439A299A64E621
:1019300070E080E090E00E94E5284398299864E6F2
:1019400070E080E090E00E94E528CF5FECCF6CE291
:1019500071E080E090E00E94E528E4CF0F931F93B0
:10196000CF93DF93EC01062F15E0115051F0CE011B
:101970000E947730081741F0602FCE010E947F301F
:10198000F4CF82E00E94910CDF91CF911F910F91D3
:101990000895A0E0B0E0EFECFCE00C945D2E482E42
:1019A000562EC0E0D0E0612C712CE12CF12C00E02F
:1019B00010E041100CC06090D40586E4689E3001B0
:1019C000112459E1E52EF12C0AEB15E01EC091E03F
:1019D00049120FC06090D405E6E46E9E30011124D8
:1019E000FBE16F0E711C49E2E42EF12C06E715E0D5
:1019F0000CC082E0481209C028E1622E772473945B
:101A0000EE24E394F12C03ED15E043018C0E9D1EB2
:101A100010927505109274053401A62CA818B12CEB
:101A2000C30101966C01AE14BF04A8F4A00EB11E50
:101A3000511006C0C3010E947730F501808305C0B4
:101A4000F5016081C3010E94AE0CF50180810E9406
:101A500061063601E2CFC301511018C0C3010E94D4
:101A60007730B82EC6010E9477302B2D30E0322F10
:101A70002227282B80917405909175058217930772
:101A800079F4C0E0D0E05524539493CF36016091AF
:101A900075050E94AE0C60917405C6010E94AE0CE3
:101AA000C05EDE4FC13E92E0D90708F482CF852D9B
:101AB000CDB7DEB7E0E10C94792E61E082E00E94C0
:101AC000C90C089560E082E00E94C90C8091D305A2
:101AD000853020F01092D3050E945D0D8091D305D2
:101AE0008093D405089561E080E00E94C90C61E014
:101AF00081E00E94C90C089560E080E00E94C90C5A
:101B0000882351F060E081E00E94C90C882321F015
:101B100080917605883349F00E94BF060E947A06BC
:101B200081E00E94DF060E94730D0895882319F05A
:101B30006AEA71E002C06EEA71E082EE95E00E940E
:101B4000AE2A0895FF920F931F93CF93DF9369EC12
:101B50007BE082EE95E00E945A2A40917B055091ED
:101B60007C0560917D0570917E052AE030E082EE73
:101B700095E00E94832B63EB7BE082EE95E00E9470
:101B80005A2A40917F05509180056091810570919E
:101B9000820520E130E082EE95E00E94832B6DE922
:101BA0007BE082EE95E00E945A2A4AE050E0609184
:101BB000830582EE95E00E94AB2B67E87BE082EE26
:101BC00095E00E945A2A4AE050E06091840582EE36
:101BD00095E00E94AB2B61E77BE082EE95E00E94EE
:101BE0005A2AC5E8D5E0F12C8E0188818823A9F016
:101BF000FF2031F061EB71E082EE95E00E947D2ADA
:101C000021964AE050E0F801608182EE95E00E9462
:101C1000742BF394F8E1FF12E7CF82EE95E00E9477
:101C2000882A6BE57BE082EE95E00E945A2A4AE022
:101C300050E060919D0582EE95E00E94AB2B66E43A
:101C40007BE082EE95E00E945A2AE0919E05E770C3
:101C5000F0E0EE0FFF1FEE57FC4F6081718182EEC6
:101C600095E00E94AE2A61E37BE082EE95E00E945F
:101C70005A2A80919E058871883069F028F4811174
:101C800013C068E27BE00CC0803141F0883161F420
:101C90006CE07BE005C06CE17BE002C066E17BE0CC
:101CA00082EE95E00E949C2A68EF7AE082EE95E051
:101CB0000E945A2A409177055091780560917905E4
:101CC00070917A052AE030E082EE95E00E94832B45
:101CD0006FED7AE082EE95E00E945A2A8091BF056E
:101CE00080710E94960D66EC7AE082EE95E00E948B
:101CF0005A2A8091BF0580740E94960D6DEA7AE0A1
:101D000082EE95E00E945A2A8091BF0580720E945F
:101D1000960D60E97AE082EE95E00E945A2A86E705
:101D200095E00E942708AB01BC012AE030E082EE7A
:101D300095E00E94652B6BE87AE082EE95E00E94C8
:101D40005A2A86E795E00E9427089B01AC0160E4CF
:101D500072E48FE090E00E941A2EBA01A9012AE0F5
:101D600030E082EE95E00E94652B68E87AE082EE32
:101D700095E00E949C2ACDB7DEB7E5E00C94842E56
:101D80008F929F92AF92BF92CF92DF92EF92FF928B
:101D9000811107C06FE77AE082EE95E00E949C2AED
:101DA0002FC090E00E94740724E630E040E050E04D
:101DB0000E941A2ECA01B9012AE030E040E050E04A
:101DC0000E941A2E49015A016B017C012AE030E081
:101DD000B501A40182EE95E00E94652B6EE282EED1
:101DE00095E00E94802A2AE030E0B701A60182EE49
:101DF00095E00E94652B63E782EE95E00E94C02A81
:101E0000FF90EF90DF90CF90BF90AF909F908F901A
:101E100008951F93CF93DF9365E77AE082EE95E014
:101E20000E945A2A80919F05813041F46CE57AE046
:101E300082EE95E00E949C2A10E050C0823019F496
:101E400065E47AE0F5CF843019F461E37AE0F0CF0D
:101E5000853091F766E27AE0EBCFC12FD0E0C93050
:101E6000D1050CF441C068E3610F82EE95E00E9459
:101E7000802A6EE17AE082EE95E00E945A2ABE0145
:101E80006F5F7F4F4AE050E082EE95E00E94442B66
:101E900063E17AE082EE95E00E945A2AC156DA4F59
:101EA000E981E03218F566E07AE082EE95E00E9482
:101EB0005A2A8981803130F06DE673E082EE95E038
:101EC0000E947D2A69816F7070E06F5F7F4F4AE0EA
:101ED00050E082EE95E00E944D2B1F5F80914805F7
:101EE000181708F4BACF0FC061E3BECFEF70F0E06F
:101EF000EE0FFF1FEE56FC4F6081718182EE95E080
:101F00000E94AE2AEACF6BEE79E082EE95E00E9465
:101F10005A2A8091B7050E94C00E60ED79E082EEEA
:101F200095E00E945A2A8091B8050E94C00E65EB88
:101F300079E082EE95E00E945A2A8091B9050E94CC
:101F4000C00E6AE979E082EE95E00E945A2A40913B
:101F5000AF055091B0056091B1057091B205411582
:101F600051056105710539F12AE030E082EE95E016
:101F70000E94832B67E679E082EE95E00E945A2A60
:101F80008091B3050E949907AB01BC012AE030E0C3
:101F900082EE95E00E94832B63E479E082EE95E087
:101FA0000E945A2A4AE050E06091B40582EE95E022
:101FB0000E94AB2B06C06AE379E082EE95E00E94B6
:101FC0009C2A6DE179E082EE95E00E945A2A6091A8
:101FD000B5057091B6054AE050E082EE95E00E94AA
:101FE000952B60E079E082EE95E00E945A2A60919C
:101FF000AE05603450F470E06F5F7F4F4AE050E010
:1020000082EE95E00E944D2B06C067EF78E082EEED
:1020100095E00E949C2A6AED78E082EE95E00E94AD
:102020005A2A8091AD0580FF03C063EB71E002C0C6
:1020300067EB71E082EE95E00E94AE2A6DEB78E0EE
:1020400082EE95E00E945A2A8091AD0582700E942E
:10205000960D6EE978E082EE95E00E945A2A809112
:10206000AD0584700E94960D6FE778E082EE95E0F2
:102070000E945A2A8091AD0588700E94960DDF91CA
:10208000CF911F9108950F931F93CF93DF932091CA
:1020900045052F3FA9F56FEF75E082EE95E00E94B0
:1020A0005A2A81E893E00E94620C6EED75E082EEA0
:1020B00095E00E945A2A80914605909147050E941A
:1020C000620C6BEA75E082EE95E00E949C2A68E85B
:1020D00075E082EE95E00E949C2A60E775E082EE52
:1020E00095E00E949C2A6BE475E082EE95E00E94E8
:1020F0009C2A82EE95E00E94882A0E94090F68C0FF
:1021000012160CF065C0332727FD309580914805E5
:1021100090E0821793070CF45BC066E375E082EEF3
:1021200095E00E945A2A60914505772767FD7095D2
:102130004AE050E082EE95E00E944D2B6BE075E0A6
:1021400082EE95E00E945A2A10E008E2809149054B
:102150001817D0F5C12FD0E0CC0FDD1FC65BDA4FCA
:10216000288130E080914505992787FD909501975A
:102170002817390739F56BEB71E082EE95E00E9484
:102180007D2A4AE050E0602F82EE95E00E94742B99
:102190006FEB71E082EE95E00E947D2AE981EF709D
:1021A000F0E0EE0FFF1FEE56FC4F6081718182EE72
:1021B00095E00E947D2A63EC71E082EE95E00E943A
:1021C0007D2A0F5F1F5FC2CF82EE95E00E94882AB2
:1021D000DF91CF911F910F910895FF920F931F935D
:1021E000CF93DF93C5E8D5E0F12C8E018881882359
:1021F000D1F165EC71E082EE95E00E947D2A4AE023
:1022000050E06F2D82EE95E00E94742B62ED71E03C
:1022100082EE95E00E947D2A2196F801208130E02F
:10222000A0E1B7E20E94D42D9B01AC01A0918405EE
:10223000B0E00E94E32DAB01BC0180917B05909141
:102240007C05A0917D05B0917E05480F591F6A1F3E
:102250007B1F2AE030E082EE95E00E94832BF3940E
:10226000F8E1FF12C2CFCDB7DEB7E5E00C94842EC3
:102270001092DF0485E6E0EEF4E0DF011D928A951E
:10228000E9F70895CF93C82F8F3719F0883009F0F8
:1022900045C0E091DF04EE23D9F1E150E093DF0483
:1022A000F0E0E052FB4F10826DE070E082EE95E0CE
:1022B0000E945906C0E08091DF04C81760F4EC2F3B
:1022C000F0E0E052FB4F608170E082EE95E00E940A
:1022D0005906CF5FF0CF60E270E082EE95E00E9499
:1022E00059066DE070E082EE95E00E945906C0E06C
:1022F0008091DF04C81778F5EC2FF0E0E052FB4F37
:10230000608170E082EE95E00E945906CF5FF0CFC9
:1023100067E082EE95E00E94802A1DC08B3119F49F
:102320000E9438111AC08D30C1F08A30B1F080910E
:10233000DF04843668F76C2F70E082EE95E00E942F
:102340005906E091DF0481E08E0F8093DF04F0E016
:10235000E052FB4FC08380E001C081E0CF9108953F
:10236000CF93C82F0E94C2286093C8047093C904F9
:102370008093CA049093CB04C093DD04CC2329F04E
:1023800040E051EE60E070E004C040E855E260E0FB
:1023900070E082EE95E00E940A2DCF910895909111
:1023A000CC04492F4F7050E0BA016F5F7F4F292F47
:1023B00030E0E4E035952795EA95E1F76217730779
:1023C00059F0FA01E353FB4F808381E0890F8F704E
:1023D000907F892B8093CC0408956EE770E082EEA5
:1023E00095E00E9459060895A3E1B1E0EAEFF1E11A
:1023F0000C945E2EE5E8F5E0712C8191882321F0A4
:10240000739428E17212F9CF66ED71E082EE95E0E7
:102410000E94AE2A4AE050E0672D82EE95E00E94CD
:10242000AB2B80E00E94B00A0E948B0B8E010E5FE6
:102430001F4FC12CD12C7601C39466246A945C2C66
:102440000E94B6284B015C012091840530E0A0E198
:10245000B7E20E94D42D9B01AC01C701B6010E94D6
:10246000F62D20917B0530917C0540917D055091A2
:102470007E05620F731F841F951F2091BB0530914D
:10248000BC054091BD055091BE052617370748078A
:10249000590718F4F80160822AC08C2D0E94E409C3
:1024A00061E070E080E090E00E94E528F801108291
:1024B0000E94B628681979098A099B09643F71400E
:1024C0008105910540F40E94FA09F801908198175E
:1024D00078F78083EDCF85B150FE05C08B7D85B93F
:1024E000439A299A04C0846285B9439829982FEFAA
:1024F000C21AD20AE20AF20A0F5F1F4F8FEFC81604
:10250000D104E104F10409F09ACFCE019395FC01C6
:10251000D82E7FEF68EC2E2F281B271510F051E0E6
:1025200056C0DE01129651E02FEF41E03D91321787
:1025300010F0322F01C0452F5F5F5F3F11F0232F56
:10254000F5CF4193242F30E0A1E0B0E0AC0FBD1FE8
:10255000A20FB31F5C93413079F0DE01A20FB31FCD
:102560005C93423049F0AFEFBFEFAC0FBD1FA20F3D
:10257000B31F6C934E3F78F6A2E0B0E0AC0FBD1FE6
:10258000A20FB31F7C934D3F30F6A3E0B0E0AC0F39
:10259000BD1FA20FB31F6C93BECF452F242F30E079
:1025A000FC01E20FF31F6081AFEFB0E0AC0FBD1F85
:1025B000A20FB31F2C91621748F44150DC01A40F05
:1025C000B11D2C9120836C934111E8CF5F5F5715AB
:1025D00020F3372D369520E0231770F4DC01A20F8D
:1025E000B11D4C91522F530FFC01E50FF11D50818D
:1025F0005C9340832E5FF0CFF5E8EF2EF5E0FF2EE1
:102600008C01802F8D19871598F4F801C1908F01E6
:102610004AE050E06C2D82EE95E00E94742B6CE253
:1026200082EE95E00E94802AF701C1927F01E9CFF6
:1026300082EE95E00E94882A81E0CD5EDE4FEFE0D9
:102640000C947A2E1F920F920FB60F9211241F93A3
:102650002F933F934F935F936F937F938F939F93AA
:10266000AF93BF93CF93DF93EF93FF93C091860017
:10267000D091870080918704909188042091A904CB
:10268000211155C09E01281B390B8091BF059091E7
:10269000C005A091C105B091C20585FD02C0369567
:1026A0002795253C49E03407B8F140910A0150E0F4
:1026B00060E070E02CE1B695A795979587952A95EF
:1026C000D1F70097A105B10521F481E090E0A0E0E9
:1026D000B0E084179507A607B707D8F480910A01E0
:1026E0008F3FB9F040E080910A01481780F4842FB1
:1026F00090E0880F991FFC01E757FB4F2081318143
:10270000FC01E55FFE4F318320834F5FECCF1092D9
:10271000AA0410920A010BC02D3B82E0380720F07A
:1027200080910A018031D8F08FEF80930A01D09315
:102730008804C0938704FF91EF91DF91CF91BF91FF
:10274000AF919F918F917F916F915F914F913F9149
:102750002F911F910F900FBE0F901F901895109101
:102760000A0181E0810F80930A01C9010E941109C9
:10277000E12FF0E0EE0FFF1FE757FB4F91838083BF
:10278000D6CF83E0809380008AE980938100809196
:10279000BF0586FD05C08091810080648093810023
:1027A0008FEF9FEF909389008093880080916F0056
:1027B000806280936F0008950E94620D8091D4051D
:1027C000843011F41092D40508956F3018F0869576
:1027D0008058089589E0689F802D11240895A0E015
:1027E000B0E0E5EFF3E10C94652EC82F0E94C228FB
:1027F000009138041091390420913A0430913B043F
:102800006B017C01C01AD10AE20AF30A9701860122
:1028100049E8C41643E1D406E104F10410F0109233
:102820003C04609338047093390480933A04909385
:102830003B042091A9048FEF820F8230D8F5E091FC
:102840003C04EE2309F44EC1E13011F482E0B8C13A
:10285000E03108F034C181E08E0F80933C04F0E059
:10286000E757FB4FC083803109F0ACC1EBE8F4E0DF
:10287000213029F4A181A695A695808108C0808188
:102880009181A92FA695A695A69596958795A03195
:1028900048F4B0E090E0AA0FBB1FA55FBE4F1196B1
:1028A0009C938E931092AA04329684E0E939F8073B
:1028B000F9F688C1233009F005C1E0913C04E1112B
:1028C00004C0CF3009F07EC10DC1E83148F481E089
:1028D0008E0F80933C04F0E0E857FB4FC08372C139
:1028E000E83109F0ECC0C111EAC040E050E0ABE0D3
:1028F000CA01B3E0880F991FBA95E1F7A49F900130
:10290000A59F300D1124F901E757FB4F6081E1814C
:102910007E2F777075956795FC01EE0FFF1FE55FC1
:10292000FE4F71836083F901E657FB4FB081B69586
:10293000B695B695E181FE2FF295FF0FF07E6F2FD1
:102940006B2BE695E695E6957E2F777075956795E6
:10295000FC01EE0FFF1FE35FFE4F71836083F901FF
:10296000E557FB4FB081B295B695B695B370C1816E
:10297000DC2FDD0FDD0F6D2F6B2BC295C695C69535
:10298000C370E281E170EE0FEE0F7E2F7C2B759508
:102990006795FC01EE0FFF1FE15FFE4F71836083BF
:1029A000F901E357FB4FB081B695E181FE2FF79512
:1029B000FF27F7956F2F6B2BE6957E2F7770759518
:1029C0006795FC01EE0FFF1FEF5EFE4F7183608382
:1029D000F901E257FB4FB081B295BF70E181FE2F44
:1029E000F295F07F6F2F6B2BE295EF707E2F777053
:1029F00075956795FC01EE0FFF1FED5EFE4F71832D
:102A00006083F901E157FB4FB081BB1FBB27BB1FA0
:102A1000C181DC2FDD0F6D2F6B2BCC1FCC27CC1F82
:102A2000E281E370EE0F7E2F7C2B75956795FC019C
:102A3000EE0FFF1FEB5EFE4F71836083F901EF56CF
:102A4000FB4FB081B695B695E181FE2FF295FF0F51
:102A5000FF0FF07C6F2F6B2BE695E6957E2F77703E
:102A600075956795FC01EE0FFF1FE95EFE4F7183C0
:102A70006083F901EE56FB4F208122952695277041
:102A80003181E32FEE0FEE0FEE0F6E2F622B732FBF
:102A900072957695777075956795FC01EE0FFF1F1F
:102AA000E75EFE4F718360834F5F5F4F4230510599
:102AB00009F01ECF80919F0483FF1092AA04109208
:102AC0003C0480C0243009F07DC060913C04611159
:102AD0000BC0C83AB1F4109275051092740588EADB
:102AE0000E94610681E06CC0613019F4C093370424
:102AF00004C0623031F4C09336048C2F0E9461060A
:102B00005AC0E09136042E2F30E0220F331F462F9B
:102B100050E0C9010296841795073CF0633268F7CC
:102B2000FA01EA57FB4FC083E8CF2D5F3F4F8C2F50
:102B300090E060917405709175054217530749F450
:102B4000982F88278627972790937505809374057B
:102B500032C06817790769F580913704813049F5EB
:102B6000E13118F080E180933604F0903604CAE831
:102B7000D4E000E010E00F15D0F4FE013197808121
:102B800090E0982F88272881822B63E0969587957F
:102B90006A95E1F70E941109F801EE0FFF1FE55F4A
:102BA000FE4F918380830F5F1F4F2296E4CF1092D8
:102BB000AA0410923C0480913C04882319F08F5F92
:102BC00080933C04CDB7DEB7E8E00C94812EE82F6B
:102BD000F0E0E654FA4FE185E03150F4F894F0E08B
:102BE000EE0FFF1FE55FFE4F80819181789408957D
:102BF000E03121F0E13131F483E101C082E10E9452
:102C0000042A089580E092E00895A2E2B0E0EBE0AB
:102C1000F6E10C945B2E9E012F5F3F4F80E1D901BE
:102C20001D928A95E9F764E072E082EE95E029A3AF
:102C30003AA30E94AE2A0E94AE0B1D8A1E8A1F8AEA
:102C4000188E312C212C00E0812C912C540170EC39
:102C5000472E7DE9572E78E5672E75E3772EE0E560
:102C6000CE2EE3ECDE2EE12CF12C84EF91E0A0E0FF
:102C7000B0E08D8F9E8FAF8FB8A380EC97EFAAEB5B
:102C8000B7E3898F9A8FAB8FBC8F80EC9DE9A8E565
:102C9000B5E3898B9A8BAB8BBC8B82EE95E00E945F
:102CA000C22B892B09F4E1C082EE95E00E94EF2B44
:102CB0009C0133272C32310509F442C0ACF4233295
:102CC000310509F0ABC019821A821B821C821D8259
:102CD0001E821F82188619861A861B861C861D86F0
:102CE0001E861F86188A60C02434310529F02335DA
:102CF000310509F4B2C092C064E482EE95E00E940E
:102D0000802A2AE030E040EC5DE968E575E382EE78
:102D100095E00E940E2B6CE282EE95E00E94802AE4
:102D20002AE030E040EC57EF6AEB77E382EE95E083
:102D30000E940E2B6CE282EE95E00E94C02AADCF7D
:102D40000F5F043009F0A9CF29813A814B815C8162
:102D5000A8EEB3E00E94E32D698B7A8B8B8B9C8B62
:102D60002D813E814F8158850E94E32D698F7A8F96
:102D70008B8F9C8F29853A854B855C852D8F3E8F67
:102D80004F8F58A32D853E854F8558890E94E32D8E
:102D90006B017C0160323EE473078105910530F4DC
:102DA00062E38CE10E94D10900E077CF603345E710
:102DB00074078105910510F462E2F3CF60345CE999
:102DC00075078105910510F466E2EBCF80E5C81622
:102DD00083ECD806E104F10410F462E1E2CF90E65E
:102DE000C9169AEED906E104F10410F465E1D9CFD1
:102DF000A0E7CA16A1E1DA06A1E0EA06F10410F4A0
:102E000061E0CFCFB0EACB16B6E8DB06B1E0EB0667
:102E1000F10410F463E0C5CF65E0C3CF10ED180FE7
:102E20001A3008F03ACFE1E0F0E0EC0FFD1F24E0AB
:102E3000029FE00DF11D11242081318142815381D7
:102E4000AAE0B0E00E94E32D610F711D811D911D6C
:102E5000608371838283938320CF49885A886B88EB
:102E60007C88812C912C540118CF81149104A104E9
:102E7000B10489F4C301B2010E94400A61E070E02C
:102E800080E090E00E94E5281D8A1E8A1F8A188E25
:102E9000312C22242A948D8D9E8DAF8DB8A1881659
:102EA0009906AA06BB06D0F40E94FA092D893E892C
:102EB0004F89588D280F311D411D511D2D8B3E8B83
:102EC0004F8B588F381608F4382E821508F4282EA8
:102ED0003FEF831A930AA30AB30A56C0C301B20193
:102EE00028EE33E040E050E00E941A2EBA01A9011A
:102EF0002AE030E082EE95E00E94652B6CE282EEE3
:102F000095E00E94802A4AE050E0632D82EE95E031
:102F10000E94742B6CE282EE95E00E94802A6D89FB
:102F20007E898F89988DA50194010E941A2EBA017D
:102F3000A9012AE030E082EE95E00E94652B6CE268
:102F400082EE95E00E94802A4AE050E0622D82EEF7
:102F500095E00E94742B6CE282EE95E00E94C02AFC
:102F60004C0C5D1C6E1C7F1C898D9A8DAB8DBC8DAD
:102F700084159505A605B70520F449885A886B88FD
:102F80007C88812C912C540129893A894B895C8950
:102F9000283E33404105510509F07FCEA296E2E17B
:102FA0000C94772EACE1B0E0E8EDF7E10C94652EDF
:102FB0000E94C2286B017C0181E00E94B00A14E7E4
:102FC00003E0198361E0CE0101960E940D0C00938D
:102FD00073050E948B0B6AEF70E080E090E00E9426
:102FE000E52880917305833089F482EE95E00E9494
:102FF000C22B892B59F40E94C2286C197D098E09B5
:103000009F096038734C894C9140D8F280917305C8
:10301000833009F44FC08FE70E94A9090E94BC09C0
:103020008983843511F083E05CC00E94BC09109252
:103030004605809347050E94BC09209146053091C2
:103040004705280F311D30934705209346050E9400
:10305000BC09809348050E94BC09809349058131D1
:1030600010F7F12C0F2D10E08091490590E0880FAA
:10307000991F0817190740F40E94BC09F801E65B84
:10308000FA4F8083F394EECF80E7898361E0CE012D
:1030900001960E940D0C83E0809373050E948B0BB8
:1030A00062E370E080E090E00E94E5288091730583
:1030B000833011F482E015C08FE70E94A9090E94B5
:1030C000BC098983803509F0AECF0FE915E00E9475
:1030D000BC09F80181938F01F5E00A3B1F07B9F79E
:1030E00081E06C96E8E00C94812E8091450599274B
:1030F00087FD9095A92FB92FFC013196EB30F10592
:1031000008F066C0EC5CFF4F0C94922E62E778E00A
:1031100082EE95E00E949C2A81E893E00E94620C76
:103120006AE578E082EE95E00E949C2A65E378E00B
:1031300082EE95E00E949C2A6BE078E082EE95E0BA
:103140000E949C2A6AEE77E082EE95E00E949C2A1B
:103150006DEB77E082EE95E00E949C2A67E977E0CC
:1031600082EE95E00E949C2A63E777E082EE95E08C
:103170000E949C2A6CE477E082EE95E00E949C2AF3
:1031800082EE95E00E94882A0E94A20D21C06FE283
:1031900077E01AC06AE077E017C065EF76E014C008
:1031A00066ED76E011C062E976E00EC06DE776E08C
:1031B0000BC068E676E082EE95E00E949C2A62E20F
:1031C00076E002C06CE076E082EE95E00E949C2AF8
:1031D0006AE070E080E090E00E94E52882EE95E0F1
:1031E0000E94C22B892B29F082EE95E00E94EF2BE2
:1031F000F5CF0895ACE1B0E0E0E0F9E10C94652E84
:10320000909145059F3F09F023C1482F50E0FA01F6
:103210003A97EF36F10508F00FC1E15CFF4F0C94CF
:10322000922E61E172E0A0C06DE172E082EE95E065
:103230000E94AE2A85E789838BE1EFE9F5E0DE01A4
:10324000129601900D928A95E1F76CE1CE010196FC
:103250000E940D0C0E948B0B83E08093730568EC39
:1032600070E080E090E00E94E52880917305843052
:1032700009F0E2C08FE70E94A9090E94BC09898376
:10328000853509F0D9C06DEE74E082EE95E00E94BC
:103290009C2A6FEC74E082EE95E00E949C2A61EB20
:1032A00074E096C065E372E082EE95E00E94AE2A7B
:1032B00089E6898361E0CE0101960E940D0C0E948F
:1032C0008B0B83E08093730568EC70E080E090E006
:1032D0000E94E52880917305843009F0ADC08FE726
:1032E0000E94A9090E94BC0989838E010E5F1F4FAD
:1032F0007E014DE1E40EF11C0E94BC09F8018193AE
:103300008F01EE15FF05C1F78BE1FE013296AFE9A3
:10331000B5E001900D928A95E1F78981893409F031
:103320008BC063E974E082EE95E00E949C2A65E719
:1033300074E082EE95E00E949C2A67E574E048C044
:103340006FE472E082EE95E00E94AE2A8EEF8093E9
:10335000450572C080528750805390914805981758
:1033600008F066C06EE572E082EE95E00E94AE2A3B
:1033700063C084E18093450560E274E029C085E183
:103380008093450569EE73E023C086E1809345058F
:1033900062EB73E01DC087E18093450568E673E04A
:1033A00017C088E18093450567E573E011C089E1A6
:1033B0008093450563E473E00BC08AE18093450583
:1033C0006EE273E005C08BE18093450566E073E033
:1033D00082EE95E00E949C2A2FC06CEE72E082EE95
:1033E00095E00E949C2A8091AD0591E01DC066ED9C
:1033F00072E082EE95E00E949C2A8091AD0592E0F9
:1034000013C061EC72E082EE95E00E949C2A8091EC
:10341000AD0594E009C066EA72E082EE95E00E9494
:103420009C2A8091AD0598E089278093AD058FEFA8
:10343000809345050E94431082EE95E00E94C22BC6
:10344000892B09F45BC182EE95E00E94EF2BF4CF4B
:103450000E944211882309F451C18091DF04811137
:1034600004C08FEF8093450541C140E050E060E02B
:1034700070E080EE94E00E94092F40914505042FF2
:10348000112707FD1095212F312FF8013197EB31CE
:10349000F10508F01BC1E255FF4F0C94922E552701
:1034A00047FD50952091480530E0241735070CF46E
:1034B0000DC18B019C010150110921093109003214
:1034C00011052105310558F0C0904905EBE4F5E000
:1034D000F12CD12CA8E2EA2E415051090FC0FA017B
:1034E000E156FA4F61506083D9C0DF0111972C91EA
:1034F00030E02417350729F0F3943296FC10F5CF0D
:10350000CBC00E2D10E020E030E00617170728078B
:10351000390741F42081DA01A156BA4F11962C9354
:10352000DD24D394E394E8CF6F3F710581059105C5
:1035300011F008F0CBC06093B705B0C06F3F7105C4
:103540008105910511F008F0C1C06093B805A6C0CF
:103550006F3F71058105910511F008F0B7C06093C8
:10356000B9059CC02091E00420622037E9F440E0D6
:1035700050E060E070E081EE94E00E94092F9B0132
:10358000AC01DC01CB010197A109B1090897A105A4
:10359000B10508F0AEC0A4EDB0E30E94E32D6A5E71
:1035A0007C4A8A46954E24C02636E9F440E050E035
:1035B00060E070E081EE94E00E94092F9B01AC0175
:1035C000DC01CB010197A109B1090797A105B1055C
:1035D00008F08FC0A8EAB1E60E94E32D645E7C4348
:1035E0008E46944E05C0611571058105910579F0EF
:1035F0008B019C01005C1D49284535430130FAE5EB
:103600001F07F2E62F07F2E03F0708F05FC0609364
:10361000AF057093B0058093B1059093B2053EC09D
:103620006F3F71058105910511F008F04FC060935F
:10363000B30534C08B019C010150110921093109E6
:103640000F3F11052105310508F040C06093B40516
:1036500025C08B019C01045C1940210931090D34FE
:103660004DE114072105310528F47093B6056093E8
:10367000B50514C0611571058105910521F48FEF21
:103680008093AE050BC06134710581059105F0F49E
:1036900061506093AE0502C0DD20C1F08091DE0470
:1036A00081111AC080917F0590918005A0918105BC
:1036B000B09182050196A11DB11D80937F05909365
:1036C0008005A0938105B093820506C060E772E093
:1036D00082EE95E00E94AE2A0E9438118FEF80930F
:1036E00045056AE082EE95E00E94C02A0E944310E0
:1036F00005C061E070E080E090E07ACF6C96E8E091
:103700000C94812E6AE572E082EE95E00E949C2A7C
:1037100062E472E082EE95E00E949C2A82EE95E0DF
:103720000E94C22B892B31F082EE95E00E94EF2B94
:103730000E94FA180E94D217823029F0833051F487
:103740006DE072E002C064E272E082EE95E00E94F9
:103750009C2A08958FEF809345051092DE040E9405
:103760004310809145058E3F69F082EE95E00E94FE
:10377000C22B892BB1F382EE95E00E94EF2B0E94C1
:10378000FA18EFCF08950F931F93109145051F3F2F
:1037900009F0D2C0893409F457C000F5883309F420
:1037A00069C058F4803309F477C008F061C08B31E8
:1037B00009F440C08132B1F1B9C0813409F487C045
:1037C00030F4893309F466C0803461F1AFC08234CB
:1037D00009F48EC0863409F448C0A8C0823609F4C2
:1037E00087C078F4883531F128F48235C1F183350A
:1037F000E1F09CC08A3509F494C0813609F467C0B1
:1038000095C0823761F128F4863679F18936E1F086
:103810008DC0883779F08A3709F483C0833709F07F
:1038200085C003C061E172E015C00E94730D6EE8AF
:1038300072E004C00E947C0D68EA72E082EE95E0BE
:103840000E94AE2A8EEF70C00E947A060E94BF06C8
:1038500067EC72E082EE95E00E94AE2A67C081E0DC
:103860000E94DF0660EE72E0F5CF0E94ED105EC0B0
:1038700080535AC06AEF71E082EE95E00E949C2A64
:1038800090919E0588E0890F8871977E892B80939F
:103890009E051AC089E048C067EE71E082EE95E0AF
:1038A0000E949C2A8091BF059091C005A091C105FE
:1038B000B091C20520E182278093BF059093C00597
:1038C000A093C105B093C205109345052FC061EDCB
:1038D00071E082EE95E00E949C2A8091BF05909154
:1038E000C005A091C105B091C20540E4842710C075
:1038F00060EC71E082EE95E00E949C2A8091BF0509
:103900009091C005A091C105B091C20520E2822727
:103910008093BF059093C005A093C105B093C205E5
:1039200002C00E94821B8FEF809345058091450560
:103930008E3F09F0D4C0DDC00E944211882309F4F3
:10394000D8C08091DF04811104C08FEF80934505BA
:10395000C6C040E050E060E070E080EE94E00E947D
:10396000092F00914505112707FD1095212F312FB3
:10397000F8013197E930F10508F0B4C0E753FF4F83
:103980000C94922E8B019C01015C1D492845354306
:103990000F3F19452246324008F0A4C060937B05D2
:1039A00070937C0580937D0590937E0577C060932E
:1039B0007F0570938005809381059093820581E057
:1039C0008093DE046BC0683071058105910508F0B5
:1039D00089C06093830562C08B019C01015011096D
:1039E000210931090A3011052105310508F07AC095
:1039F0006093840553C061EB71E080EE94E00E9417
:103A0000433010E0009799F00E941D30009779F044
:103A1000183130F4E12FF0E0EA58FA4F87871F5F42
:103A200061EB71E080E090E00E944330EBCF183111
:103A3000A8F5E12FF0E0EA58FA4F17861F5FF7CF9D
:103A4000653071058105910508F04CC060939D05B6
:103A500025C08B019C010150110921093109063053
:103A6000110521053105F0F520919E05287F262BB3
:103A700020939E0513C08B019C010150110921095F
:103A800031090115124C2140310560F5609377052D
:103A9000709378058093790590937A058091DE0480
:103AA000811113C080917F0590918005A0918105BF
:103AB000B09182050196A11DB11D80937F05909361
:103AC0008005A0938105B09382050E9438118FEF85
:103AD000809345056AE082EE95E00E94C02A0E942C
:103AE000751807C060E772E082EE95E00E94AE2A8A
:103AF000ECCF1F910F9108958FEF809345051092A1
:103B0000DE040E947518809145058E3F69F082EEB3
:103B100095E00E94C22B892BB1F382EE95E00E94C2
:103B2000EF2B0E94C31BEFCF6AE070E080E090E0D3
:103B30000E94E52882EE95E00E94C22B892B29F095
:103B400082EE95E00E94EF2BF5CF0895CF93C82F1A
:103B5000682F82EE95E00E941C2C90916A059C27AC
:103B600090936A05CF910895A1E0B0E0EAEBFDE102
:103B70000C946B2E99830E94A61D9981892F0E9417
:103B8000A61D2196E2E00C94872E1F93CF93DF931E
:103B9000182FEB0110926A0565EB70E082EE95E05C
:103BA0000E94590662E670E082EE95E00E94590696
:103BB000812F0E94A61DCE010E94B41DDF91CF91DE
:103BC0001F91089560916A0582EE95E00E941C2C79
:103BD0000895A1E2B0E0EFEEFDE10C94672E7B01C9
:103BE0008A018C3009F453C108F040C0863009F4D2
:103BF000BCC018F5833009F491C070F4813009F429
:103C000072C0823009F048C26BE170E082E00E942D
:103C1000C51D0FE915E078C0843009F487C08530F0
:103C200009F03AC26091490570E0660F771F85E0A0
:103C30000E94C51D0AE415E086C0893009F4A7C0BA
:103C400070F4873009F49BC0883009F025C261E028
:103C500070E088E00E94C51D8091D40523C28A309F
:103C600009F4CAC08B3009F4F2C016C28A3609F4CE
:103C700075C1D8F4873609F43AC138F4853609F4A9
:103C80000EC1863609F41FC107C2883609F437C150
:103C9000893609F001C261E070E089E60E94C51D25
:103CA0000E947A060E94BF06F5C18D3609F4D4C180
:103CB00038F48B3609F491C18C3609F49AC1ECC101
:103CC0008E3609F4DCC1873C09F0E6C161E070E0A2
:103CD00087EC0E94C51D81E00E94A61D0E94E21D86
:103CE00010926B05E3C169E270E081E00E94C51D9E
:103CF00006E715E0F80181918F010E94A61DF5E00D
:103D00000F391F07B9F7D0C1F80181918F010E94C7
:103D1000A61DF5E00A3B1F07B9F7C6C161E070E0D8
:103D200083E00E94C51D0E94D217BCC161E070E013
:103D300084E00E94C51D81E00E94A61D0E94E21D34
:103D40000E940516B3C18091490590E0880F991F24
:103D500098012A5435402817390708F0A5C1F80101
:103D600081918F010E94A61DEECF62E070E086E097
:103D70000E94C51D81E893E00E94B41D95C161E0D9
:103D800070E087E00E94C51D809148058BC186E6E2
:103D9000898361E0CE0101960E940D0C0E948B0B7D
:103DA00083E08093730568EC70E080E090E00E940F
:103DB000E528809173058430D9F48FE70E94A90922
:103DC0000E94BC098983863469F460E270E089E06E
:103DD0000E94C51D10E20E94BC090E94A61D115040
:103DE000D1F762C161E070E089E00E94C51D52C157
:103DF00061E070E089E053C169E170E08AE00E940F
:103E0000C51D82E08093BA05209172058091BF059F
:103E10009091C005A091C105B091C205222311F077
:103E2000806801C08F778093BF059093C005A093F1
:103E3000C105B093C2050AEB15E0F80181918F012D
:103E40000E94A61DF5E0033D1F07B9F72DC161E2F1
:103E500070E08BE00E94C51D8091AA048F3F39F06D
:103E60008091AA0491E0980F9093AA0402C08091D7
:103E7000AA040E94A61D10E0812F0E94E7150E944F
:103E80003C090E94B41D1F5F1031B1F70DC161E004
:103E900070E08CE00E94C51D8091D30503C161E0F4
:103EA00070E085E60E94C51D89E2E816F10409F07C
:103EB000F8C0D801E6E7F5E08D91819385E0EF3910
:103EC000F807D1F7E7C061E070E086E60E94C51D03
:103ED000EBE1EE16F10409F0E4C0D801EFE9F5E0FA
:103EE0008D91819385E0EA3BF807D1F7D3C061E07B
:103EF00070E087E60E94C51D0E94730DCBC061E093
:103F000070E088E60E94C51D85E789838BE1EFE9B3
:103F1000F5E0DE01129601900D928A95E1F76CE1D1
:103F2000CE0101960E940D0C0E948B0B83E08093C2
:103F3000730560E273E080E090E00E94E5288091E4
:103F40007305843009F0ADC08FE70E94A9090E9473
:103F5000BC098983853509F0A4C09CC061E070E08C
:103F60008AE60E94C51D89E6898361E0CE0101963B
:103F70000E940D0C0E948B0B83E08093730560E21E
:103F800073E080E090E00E94E52880917305843022
:103F900009F087C08FE70E94A9090E94BC098983A4
:103FA0008E010E5F1F4F7E01EDE1EE0EF11C0E94AF
:103FB000BC09F80181938F01EE15FF05C1F78BE174
:103FC000FE013296AFE9B5E001900D928A95E1F7D6
:103FD0008981893409F065C05DC061E070E08BE6DD
:103FE0000E94C51DF80180818093D4050E947C0D3C
:103FF00051C061E070E08CE60E94C51DF0E2EF1652
:10400000F10461F487E6898380E2F801DE0112960B
:1040100001900D928A95E1F761E203C087E48983FC
:1040200061E0CE0101960E940D0C0E948B0B83E093
:10403000809373056CE474E080E090E00E94E528D2
:1040400080917305843069F58FE70E94A9090E9469
:10405000BC09873431F51EC061E070E08DE60E9436
:10406000C51D89E1E816F104E1F4D801EAEBF5E0B9
:104070008D91819385E0E33DF807D1F70BC061E0B6
:1040800070E08EE60E94C51DF80180818093D30503
:104090000E945D0D81E006C061E070E08AEC0E9444
:1040A000C51D80E00E94A61D0E94E21DA196E6E0CB
:1040B0000C94832EA0E0B0E0E0E6F0E20C94652ED4
:1040C000CAECD3E014E606E035E0F32E44E0E42E3B
:1040D00053E0D52E62E0C62E82EE95E00E94C22B00
:1040E000892B09F49BC082EE95E00E94EF2B282FCC
:1040F000809335044091340450E04730510560F717
:10410000FA01EE52FF4F0C94922E853B29F781E085
:1041100080933404E1CF823609F07DC0C09234042C
:10412000DBCF8093330480933204D0923404D4CF15
:104130009C01332730933104209330049091320452
:10414000982790933204E0923404C6CF382F222768
:104150004091300450913104242B352B309331049D
:104160002093300490913204982790933204F09277
:1041700034042536310508F4AFCF61E070E08CECF3
:104180000E94C51D81E00E94A61D0E94E21D43C041
:1041900020912E0430912F04F901E653FC4F8083C7
:1041A00090913204982790933204C901019690931C
:1041B0002F0480932E042091300430913104821713
:1041C000930708F489CF0093340486CF809132049A
:1041D00082130BC060912E0470912F044AEC53E0BF
:1041E000809133040E94E91D0DC062E070E08BEC09
:1041F0000E94C51D809133040E94A61D80916A050E
:104200000E94A61DFE01812F11928A95E9F7109256
:104210002F0410922E04109234045ECFCDB7DEB777
:10422000E8E00C94812E81E080936B0580916B0512
:10423000882349F082EE95E00E94C22B892BB1F3CE
:104240000E945A20F3CF0895AAE2B0E0EAE2F1E238
:104250000C94632E0E94B6286B017C0181E00E94C1
:10426000B00A82EE95E00E94C22B892B29F082EEE3
:1042700095E00E94EF2BF5CF4398299811E072E664
:10428000B72EE9E2AE2E03E00E94B6286C197D0934
:104290008E099F09693C710581059105F0F1112393
:1042A000E1F10E94B6286B017C0185B1846285B979
:1042B00080ED97E00E94B607B982E6E7F5E0DE01FF
:1042C00012968A2D01900D928A95E1F76AE2CE014D
:1042D00001960E940D0C85B18B7D85B980E090E040
:1042E0000E94B607009373050E948B0B62E370E097
:1042F00080E090E00E94E52880917305843061F4AD
:10430000009373058FE70E94A9090E94BC0911E080
:10431000823419F410E001C011E087E00E94DB292B
:10432000892BB1F411E014C0439A299A85B18462B3
:1043300085B982EE95E00E94EF2B8D309105C1F09A
:1043400074F40A97A9F04398299885B18B7D85B9B3
:1043500082EE95E00E94C22B892B31F795CF8332F4
:10436000910579F08234910571F70E941321EBCF0A
:1043700062EB71E082EE95E00E949C2A0E947C1D17
:10438000E2CF0E940516DFCF8F929F92AF92BF922D
:10439000CF92DF92EF92FF921F93CF93DF9387E04C
:1043A0000E94DB29892B09F089C068EC70E080E06D
:1043B00090E00E94E52880E090E00E94B6070E940D
:1043C000B6284B015C016B017C0180ECC80E82E1D8
:1043D000D81EE11CF11C0E94B6286C157D058E05C7
:1043E0009F0530F487E00E94DB29892BA1F364C08C
:1043F00087E00E94DB29892B09F05EC080ED97E001
:104400000E94B6070E94B6286B017C01D0E0C1E093
:1044100088E4880E86E2981EA11CB11C11E087E09A
:104420000E94DB29892B21F58C149D04AE04BF0466
:1044300030F480ED97E00E94B607D1E0F0CF0E9403
:10444000B6286C197D098E099F09693C71058105A3
:10445000910528F30E94B6286B017C01C12719F051
:1044600080ED97E002C080E090E00E94B607D7CFD1
:1044700080E090E00E94B607DD23B9F08091D3057B
:1044800090E0019665E070E00E94062E8093D305CF
:104490000E945D0D0E94DC130E947C0D64EF71E0B0
:1044A00080E090E00E94E52809C080E00E94DF06DD
:1044B0000E94F4110E94730D0E942421DF91CF917C
:1044C0001F91FF90EF90DF90CF90BF90AF909F90A3
:1044D0008F900895CF92DF92EF92FF9280E00E943A
:1044E0000D080E94E40761E081E10E946F2961E00C
:1044F0008DE00E946F2961E089E00E946F2961E0F0
:104500008AE00E946F2960E087E00E946F2960E0E6
:1045100088E00E946F2961E088E00E94A8290E943B
:104520009F0740E052EC61E070E082EE95E00E946F
:104530000A2D0E94DC130E947C0D0E94C1138FEF94
:104540008093AA040E94F90778940E94B6286B0110
:104550007C018091AA048F3F59F40E94B6286C19FF
:104560007D098E099F09603D77408105910588F39B
:1045700080ED97E00E94B60761E087E00E94A829DD
:10458000439A299A82EE95E00E94C22B892B29F04A
:1045900082EE95E00E94EF2BF5CF6DEF72E082EE98
:1045A00095E00E947D2A81E893E00E94620C64E11C
:1045B00073E082EE95E00E947D2A4AE050E063E0DD
:1045C00070E082EE95E00E944D2B62E370E080E0A7
:1045D00090E00E94E52882EE95E00E94C22B0497AD
:1045E0000CF182EE95E00E94EF2B82349105D1F41C
:1045F00082EE95E00E94EF2B8E34910599F482EEC5
:1046000095E00E94EF2B8434910561F482EE95E0F1
:104610000E94EF2B819731F480E090E00E94B60772
:104620000E94242140917705509178056091790589
:1046300070917A05DB01CA010197A109B1090497BC
:10464000A105B10568F44093A904433029F440EA78
:1046500056E861E070E004C040E052EC61E070E0D8
:1046600082EE95E00E940A2D0E94C4214398299869
:1046700080E090E00E94B6070E94C1131092C5042A
:104680008091BF0583FF11C080918B05882351F075
:1046900080919205882331F080919905882311F04B
:1046A00087E001C085E08093C50480E00E94B00AE5
:1046B0008091C6040E94E4090E948B0B10923F0473
:1046C00010923E0410923D04F12C8091D4058F1578
:1046D000B0F062E370E080E090E00E94E52880EDB9
:1046E00097E00E94B60762E370E080E090E00E94ED
:1046F000E52880E090E00E94B607F394E6CF809131
:104700009E0584FF08C0982F987181E0983109F0C8
:1047100080E00E94B0118FE00E940D08FF90EF90A2
:10472000DF90CF900895EF92FF920F931F93CF9356
:10473000DF938C016EE770E082EE95E00E945906EF
:10474000E801F12CF0E2EF2E8E0188818D57823046
:1047500048F46DE770E082EE95E00E94590688818A
:104760008E2588832196F801608182EE95E00E9473
:104770001C2CF394F9E0FF12E7CF6EE770E082EEB5
:1047800095E00E945906CDB7DEB7E6E00C94832E83
:10479000A9E0B0E0EEECF3E20C946B2E9091C7042C
:1047A00091110EC09EEF99838A836B8350E05595DB
:1047B00047954C832D83198618861F821E822EC032
:1047C0004091CC04842F90E0B4E095958795BA95FC
:1047D000E1F7242F2F7030E08217930719F18DEF46
:1047E00089831B82FE01349650E0842F90E0A4E080
:1047F00095958795AA95E1F7242F2F7030E08217C1
:10480000930749F0DC01A353BB4F8C918193405F28
:104810005F5F563051F74093CC045A83CE01019626
:104820000E9493238091C70490E0019666E070E0B7
:104830000E94062E8093C7042996E2E00C94872EEE
:10484000A0E0B0E0E6E2F4E20C94642E6C016EE7C6
:1048500070E082EE95E00E9459068601E12CF12C71
:10486000C0E0D0E030E2B32EF801608183E8860F2B
:10487000823078F46DE770E082EE95E00E94590690
:10488000F80160816B2570E082EE95E00E94590688
:1048900004C082EE95E00E941C2CE114F10459F052
:1048A000F80180819E01280F311DC901C92FDD2724
:1048B000C80FD91FDD273FEFE31AF30A89E0E81696
:1048C000F10459F028E0E216F10421F48C2F8095D0
:1048D000F60180870F5F1F4FC7CFCDB7DEB7E9E086
:1048E0000C94802EA9E0B0E0E8E7F4E20C946B2E83
:1048F000E82F362F8091C70490E0019664E270E0C3
:104900000E94062E8093C70458E9598350E15A83C8
:10491000813089F048F08230B9F08330D9F48B834C
:1049200081EF8C833D8319C085E08B8381EF8C837D
:104930002F5F2D8312C08B8381EF8C8384E6489F89
:10494000A00111245D8309C084E08B8381EF8C83F7
:10495000ED8303C00E94ED1104C0CE0101960E94B8
:1049600020242996E2E00C94872EA2E0B0E0EBEB45
:10497000F4E20C94602E182F762E2A8349830E942D
:10498000C2286B017C018091DD048090C804909066
:10499000C904A090CA04B090CB042A81498188231D
:1049A000C1F0D701C60188199909AA09BB094C01B0
:1049B0005D0191EE89169EE29906A104B10420F1F1
:1049C000241708F4422F202F672D812F0E94722474
:1049D00013C0D701C60188199909AA09BB094C015E
:1049E0005D0191E3891695E79906A104B10460F091
:1049F000672D812F0E94C823C092C804D092C90499
:104A0000E092CA04F092CB042296EDE00C947C2E46
:104A1000A2E2B0E0EEE0F5E20C94612E8CE00E94A0
:104A2000CB0981110FC06CE173E082EE95E00E942A
:104A3000AE2A439A299A80E00E94B00A0E948B0B0A
:104A40004398299882EE95E00E94C22B892B01F1B0
:104A500082EE95E00E94EF2B9091A904992319F022
:104A60000E94EF13EFCF40913E0450E09A012F5F78
:104A70003F4F2F71332760913F0470E026173707AF
:104A800009F3FA01E75BFB4F808320933E04DACF02
:104A900080917305843009F086C00E94C228611598
:104AA00071058105910549F06093B7047093B804CE
:104AB0008093B9049093BA040CC081E090E0A0E028
:104AC000B0E08093B7049093B804A093B904B09376
:104AD000BA048091AD049091AE0481609093AE04CD
:104AE0008093AD0483E0809373058FE70E94A9094A
:104AF00009E614E00E94BC09F80181938F01F4E0FB
:104B000002371F07B9F72091720480916904982F2A
:104B1000922796FF3BC090E4922790937204982FBF
:104B200098739833F1F410E0212F30E080916904FC
:104B3000877090E0821793074CF11F5F20919E05CC
:104B4000812F90E0FC01E759FB4F24FF04C08081D6
:104B50000E94CF11E9CF608182EE95E00E941C2C6B
:104B6000E3CF8F7399F480916A048093B6048091A7
:104B70006B048093B40480916C048093B30480919F
:104B80006F0490E09093AC048093AB0480913D045B
:104B9000813019F482E080933D0480913D0483309C
:104BA00011F410923D040E94C2286B017C01809197
:104BB000AF049091B004A091B104B091B2040097F9
:104BC000A105B105C9F0A7019601281B390B4A0BB5
:104BD0005B0BDA01C901883B9B40A105B10560F080
:104BE0000E94FA098093B5041092AF041092B004A9
:104BF0001092B1041092B2048091BB049091BC0455
:104C0000A091BD04B091BE0446015701881A990ACB
:104C1000AA0ABB0A86E795E00E942708861697062F
:104C2000A806B90608F4AAC0C092BB04D092BC047E
:104C3000E092BD04F092BE040E9457068091AA043F
:104C40008830A0F08091BF059091C005A091C1056A
:104C5000B091C2056CE1B695A795979587956A9531
:104C6000D1F7892B8A2B8B2B09F0AAC18091AA043A
:104C70008F5F8093AA048091B7049091B804A091AB
:104C8000B904B091BA040097A105B105F1F0C81AB2
:104C9000D90AEA0AFB0A86E795E00E9427086C1504
:104CA0007D058E059F0508F00AC18091BF0584FD32
:104CB00004C080ED97E00E94B6071092B7041092EE
:104CC000B8041092B9041092BA0490917204907CC6
:104CD0009093720450913E0480913F0420913D04D2
:104CE000581709F409C1223009F006C19058909371
:104CF0007204E0919E05E770F0E0E658FC4F608199
:104D0000693008F0E1C0615040E04613DFC0809395
:104D10003F0487E3840F90917204892B809372047F
:104D20004093400483E080933D0485B1846285B95B
:104D3000809183059091C504911133C10E94AB0A03
:104D40008091C6040E94E409E0919E05E770F0E0BE
:104D5000E658FC4F608182E794E00E94C60BE09128
:104D6000C604EF5FE093C604E83109F426C1F0E021
:104D7000EA58FA4F8785882309F41FC10E94350C31
:104D8000813069F580919E05887149F18091AD046B
:104D90009091AE04880F991F9093AE048093AD0458
:104DA00083E0809373050E948B0B0E94C22860935E
:104DB000AF047093B0048093B1049093B204672B56
:104DC000682B692B61F481E090E0A0E0B0E0809373
:104DD000AF049093B004A093B104B093B204809157
:104DE0009E0584FF1FC08091AD049091AE048E7F1C
:104DF0000E945D09182F6091AB048091B6040E9457
:104E0000E513482F612F8091B50449A30E94E51353
:104E10000091D405282F49A16091B3048091B40476
:104E20000E94B52485B18B7D85B98091C304813002
:104E3000C1F018F08230B1F1D1C087E00E94DB29C7
:104E4000892B09F0CBC081E08093C3040E94B6286F
:104E50006093BF047093C0048093C1049093C20414
:104E6000BDC087E00E94DB29892B31F50E94B6285E
:104E7000C090BF04D090C004E090C104F090C20480
:104E80006C197D098E099F09693E73408105910562
:104E900008F4A4C082E08093C30480ED97E00E94F0
:104EA000B6079CC087E00E94DB29892B09F496C0D5
:104EB00080E090E00E94B6071092C3048FC080E0AB
:104EC00090E00E94B60701CF68E01ECF851709F475
:104ED0001ECF4F5F242F30E090E0F901EE58FB4FDA
:104EE000DC01A75BBB4F7C917083F901E05CFB4F59
:104EF000708301968F7109CF2430B1F42091400462
:104F000081E494E0A3E7B4E0FC013E2F381B3217A4
:104F100018F431913D93F9CF87E3820F9091720499
:104F2000892B80937204FECE8091C304823071F489
:104F3000916090937204439A299A53ECE52E55E0C0
:104F4000F52E8E010F5F1F4FB80111C043982998AD
:104F500080913D04811103C081E080933D048091E4
:104F60003D04833051F784E080933D04E6CFF701A0
:104F700081917F0169A37AA30E94E715F8018193CB
:104F800091938F0169A17AA1F3EDEF16F5E0FF0689
:104F900071F780919E0543E754E087700E94AC084A
:104FA000C4CE882309F4CACE2091C40431E0320F64
:104FB0003093C4042913C2CE0DC01092C604DECEB5
:104FC0008091AA04883011F4439A299A89E0809349
:104FD000AA04D4CE1092C4048150B0CEA296ECE0C4
:104FE0000C947D2E8230E8F4E82FF0E0EE0FFF1FE6
:104FF000EB52FA4F71836083813041F080916900F8
:105000008C7F842B80936900E89A089580916900D1
:10501000440F551F440F551F837F842B80936900D5
:10502000E99A08951F920F920FB60F9211242F93B1
:105030003F934F935F936F937F938F939F93AF9320
:10504000BF93EF93FF938091D5059091D605892B5F
:1050500029F0E091D505F091D6050995FF91EF91E2
:10506000BF91AF919F918F917F916F915F914F9180
:105070003F912F910F900FBE0F901F9018951F9288
:105080000F920FB60F9211242F933F934F935F937C
:105090006F937F938F939F93AF93BF93EF93FF9300
:1050A0008091D7059091D805892B29F0E091D705FB
:1050B000F091D8050995FF91EF91BF91AF919F9124
:1050C0008F917F916F915F914F913F912F910F90B1
:1050D0000FBE0F901F9018951F920F920FB60F9250
:1050E00011242F933F938F939F93AF93BF938091FE
:1050F000DA059091DB05A091DC05B091DD053091DA
:10510000D90523E0230F2D3720F40196A11DB11DF1
:1051100005C026E8230F0296A11DB11D2093D905D5
:105120008093DA059093DB05A093DC05B093DD0551
:105130008091DE059091DF05A091E005B091E10539
:105140000196A11DB11D8093DE059093DF05A0930C
:10515000E005B093E105BF91AF919F918F913F9191
:105160002F910F900FBE0F901F9018952FB7F894A6
:105170006091DA057091DB058091DC059091DD0589
:105180002FBF08953FB7F8948091DE059091DF0519
:10519000A091E005B091E10526B5A89B05C02F3F81
:1051A00019F00196A11DB11D3FBF6627782F892FE9
:1051B0009A2F620F711D811D911D42E0660F771FAE
:1051C000881F991F4A95D1F70895CF92DF92EF92E9
:1051D000FF92CF93DF936B017C010E94C228EB0109
:1051E000C114D104E104F10479F00E94C2286C1BBF
:1051F0007D0B683E7340A0F381E0C81AD108E10836
:10520000F108C851DC4FECCFDF91CF91FF90EF90C8
:10521000DF90CF900895789484B5826084BD84B582
:10522000816084BD85B5826085BD85B5816085BDA1
:10523000EEE6F0E0808181608083E1E8F0E01082BA
:10524000808182608083808181608083E0E8F0E0FB
:10525000808181608083E1EBF0E0808184608083E5
:10526000E0EBF0E0808181608083EAE7F0E080811C
:10527000846080838081826080838081816080837C
:105280008081806880831092C1000895833081F00E
:1052900028F4813099F08230A1F008958630A9F089
:1052A0008730B9F08430D1F4809180008F7D03C0C5
:1052B000809180008F7780938000089584B58F77E8
:1052C00002C084B58F7D84BD08958091B0008F7732
:1052D00003C08091B0008F7D8093B0000895CF937C
:1052E000DF9390E0FC01ED50F44F2491FC01E95F65
:1052F000F34F8491882349F190E0880F991FFC01B6
:10530000E15DF34FA591B4918B5D934FFC01C59185
:10531000D4919FB7611108C0F8948C912095822395
:105320008C93888182230AC0623051F4F8948C9166
:10533000322F309583238C938881822B888304C0FD
:10534000F8948C91822B8C939FBFDF91CF9108951D
:10535000A1E0B0E0EEEAF9E20C94692E282F30E0EB
:10536000F901E152F44F8491F901ED50F44F149199
:10537000F901E95FF34F04910023C9F0882321F07C
:1053800069830E9446296981E02FF0E0EE0FFF1F3C
:10539000EB5DF34FA591B4919FB7F8948C91611197
:1053A00003C01095812301C0812B8C939FBF219650
:1053B000E4E00C94852ECF93DF93282F30E0F901A1
:1053C000E152F44F8491F901ED50F44FD491F90179
:1053D000E95FF34FC491CC2391F081110E944629DB
:1053E000EC2FF0E0EE0FFF1FE55EF34FA591B491B7
:1053F0002C912D2381E090E021F480E002C080E038
:1054000090E0DF91CF9108958E3008F08E50877034
:1054100020919D0190E4299F90011124822B80937B
:105420007C0080917A00806480937A0080917A0079
:1054300086FDFCCF809178002091790090E0922B3E
:105440000895A0E0B0E0E7E2FAE20C94652E6C016A
:105450007A01EB01E60EF71E00E010E0CE15DF0545
:1054600061F06991D601ED91FC910190F081E02D00
:10547000C6010995080F191FF1CFC801CDB7DEB7D6
:10548000E8E00C94812E6115710589F0DB010D9027
:105490000020E9F7AD0141505109461B570BDC01D3
:1054A000ED91FC910280F381E02D0995089580E053
:1054B00090E00895EF92FF920F931F93CF93DF93A5
:1054C0008C01FB01C0E0D0E064917F018FEFE81A0E
:1054D000F80A662361F0D801ED91FC910190F0810A
:1054E000E02DC8010995C80FD91FF701EDCFCE01F6
:1054F000CDB7DEB7E6E00C94832E0E94432A0895D0
:10550000DC01ED91FC910190F081E02D0995089569
:105510000F931F93CF93DF93EC016DE00E94802ADD
:105520008C016AE0CE010E94802A800F911FDF91DA
:10553000CF911F910F9108950F931F93CF93DF93F6
:10554000EC010E945A2A8C01CE010E94882A800F09
:10555000911FDF91CF911F910F9108950F931F938A
:10556000CF93DF93EC010E94432A8C01CE010E946D
:10557000882A800F911FDF91CF911F910F9108957D
:105580000F931F93CF93DF93EC010E94802A8C012D
:10559000CE010E94882A800F911FDF91CF911F9129
:1055A0000F910895A1E2B0E0E8EDFAE20C94612ECB
:1055B0007C01C42EE52FCB01D22E19A221E02D159E
:1055C00010F02AE0D22E8E010F5D1F4F8D2C912CF2
:1055D000A12CB12C6C2D7E2FA50194010E941A2EB6
:1055E0008C2DD29E80191124015011098A3010F49B
:1055F000805D01C0895CF80180832115310541057A
:10560000510521F0C22EE32FCA01E4CFB801C70132
:105610000E94432AA196ECE00C947D2EA0E0B0E01D
:10562000E4E1FBE20C94652EEC016A017B0121159B
:10563000310541F4E881F9810190F081E02D642F7A
:1056400009951DC02A303105A9F477FF12C06DE21B
:105650000E94802A8C0144275527BA014C195D0904
:105660006E097F092AE0CE010E94D22A800F911F85
:1056700006C02AE0B701A601CE010E94D22ACDB70A
:10568000DEB7E8E00C94812E9A01AB01662757FD46
:105690006095762F0E940E2B08950F931F93CF9342
:1056A000DF93EC019A01AB01662757FD6095762FD9
:1056B0000E940E2B8C01CE010E94882A800F911F20
:1056C000DF91CF911F910F9108952115310549F474
:1056D000DC01ED91FC910190F081E02D642F0995A2
:1056E00008950E94D22A08959A01462F50E060E062
:1056F00070E00E94652B08959A01AB0160E070E0B4
:105700000E94652B08950F931F93CF93DF93EC01B5
:105710000E94652B8C01CE010E94882A800F911F68
:10572000DF91CF911F910F9108950F931F93CF9306
:10573000DF93EC019A01AB0160E070E00E94652B01
:105740008C01CE010E94882A800F911FDF91CF919A
:105750001F910F9108950F931F93CF93DF93EC0147
:105760009A01462F50E060E070E00E94652B8C01AA
:10577000CE010E94882A800F911FDF91CF911F9147
:105780000F910895FC0124853585F901E05CFF4FF8
:1057900080819181F901EE5BFF4F20813181821B75
:1057A000930B8F7399270895FC0184859585FC01DF
:1057B000E05CFF4F40815181FC01EE5BFF4F208197
:1057C00031814217530741F00190F081E02DE80F3D
:1057D000F91F808190E008958FEF9FEF0895FC01FD
:1057E00084859585FC01E05CFF4F40815181FC017F
:1057F000EE5BFF4F208131814217530779F0A08182
:10580000B181A80FB91F8C91208131812F5F3F4F4B
:105810002F7333273183208390E008958FEF9FEF1C
:105820000895FC0181A1882329F0A489B5898C9170
:1058300086FFFBCF11A20895CF93DF93FC0126854D
:105840003785D901A05CBF4F8D919C91119701962E
:105850008F739927E901CE5BDF4F48815981841707
:105860009507D9F30D90BC91A02DA20FB31F6C9397
:10587000A685B785A05CBF4F11969C938E93A68991
:10588000B7892C9181E090E0078C02C0880F991FA6
:105890000A94E2F7282B2C9381E081A30488F589F0
:1058A000E02D80818064808381E090E0DF91CF9162
:1058B000089508951F920F920FB60F9211242F93FF
:1058C0003F934F938F939F93EF93FF938091C000EB
:1058D00082FD1CC04091C600809188069091890687
:1058E00001968F73992720918A0630918B06821733
:1058F000930771F0E0918806F0918906E85BF94F13
:105900004083909389068093880602C08091C600E8
:10591000FF91EF919F918F914F913F912F910F9018
:105920000FBE0F901F90189582EE95E00E94C22B3B
:10593000892B11F00E94592C08951F920F920FB6D7
:105940000F9211242F933F938F939F93EF93FF9385
:105950002091440630914506809146069091470675
:105960002817390731F48091C1008F7D8093C100E1
:1059700014C0E0914606F0914706EC5FF94F208194
:10598000809146069091470601968F7399279093D0
:105990004706809346062093C600FF91EF919F91A2
:1059A0008F913F912F910F900FBE0F901F901895E0
:1059B000A0E0B0E0EEEDFCE20C94612EFC0113825D
:1059C000128288EE93E0A0E0B0E084839583A68302
:1059D000B7838CEB93E091838083758764875787C7
:1059E0004687318B208B138B028BF58AE48AD78A0A
:1059F000C68AB18EA08E938E828E8F85848F888981
:105A0000858F8989868F8A89878F8B8980A3ECE02F
:105A10000C947D2ECF92DF92EF92FF92CF93DF9383
:105A2000EC016A017B01411581EE580761057105A2
:105A3000F9F0EC89FD8981E090E008A002C0880FB0
:105A4000991F0A94E2F7808360E079E08DE390E0AB
:105A5000A70196010E941A2E2150310941095109CE
:105A60005695479537952795211580E1380798F089
:105A7000EC89FD89108260E874E88EE190E0A7016E
:105A800096010E941A2E215031094109510956955B
:105A9000479537952795E889F9893083EA89FB8905
:105AA000208319A2EE89FF89408181E090E09C016A
:105AB0000C8C02C0220F331F0A94E2F7422B408362
:105AC000EE89FF8940819C010D8C02C0220F331F9B
:105AD0000A94E2F7422B4083EE89FF8940819C01C2
:105AE0000E8C02C0220F331F0A94E2F7422B408330
:105AF000EE89FF8920810F8C02C0880F991F0A94BC
:105B0000E2F7809582238083DF91CF91FF90EF9021
:105B1000DF90CF9008958F929F92AF92BF92CF92D5
:105B2000DF92EF92FF920F931F9381E08F9385E0B6
:105B30008F9387E08F9383E08F9384E08F93E6ECDD
:105B40008E2E912CF2ECAF2EB12CA1ECCA2ED12CC2
:105B5000B0ECEB2EF12C04EC10E025EC30E044E04E
:105B600056E068E476E082EE95E00E94D82C0F9033
:105B70000F900F900F900F901F910F91FF90EF904B
:105B8000DF90CF90BF90AF909F908F9008950E942C
:105B90000B290E946A22C4E9DCE20E9408252097B2
:105BA000E1F30E94942CF9CFA29FB001B39FC001F2
:105BB000A39F700D811D1124911DB29F700D811D39
:105BC0001124911D08950E94D42DA59F900DB49F7E
:105BD000900DA49F800D911D11240895B7FF0C9482
:105BE000E32D0E94E32D821B930B0895DB018F931D
:105BF0009F930E94E32DBF91AF91A29F800D911DB5
:105C0000A39F900DB29F900D1124089597FB072E2E
:105C100016F4009407D077FD09D00E94982E07FC57
:105C200005D03EF4909581959F4F089570956195AC
:105C30007F4F0895A1E21A2EAA1BBB1BFD010DC0C8
:105C4000AA1FBB1FEE1FFF1FA217B307E407F5072C
:105C500020F0A21BB30BE40BF50B661F771F881F08
:105C6000991F1A9469F760957095809590959B019E
:105C7000AC01BD01CF010895052E97FB1EF40094E1
:105C80000E94532E57FD07D00E941A2E07FC03D006
:105C90004EF40C94532E50954095309521953F4FDE
:105CA0004F4F5F4F089590958095709561957F4F08
:105CB0008F4F9F4F08952F923F924F925F926F9216
:105CC0007F928F929F92AF92BF92CF92DF92EF928C
:105CD000FF920F931F93CF93DF93CDB7DEB7CA1B0D
:105CE000DB0B0FB6F894DEBF0FBECDBF09942A8838
:105CF000398848885F846E847D848C849B84AA84E0
:105D0000B984C884DF80EE80FD800C811B81AA816C
:105D1000B981CE0FD11D0FB6F894DEBF0FBECDBF37
:105D2000ED010895EE0FFF1F0590F491E02D099409
:105D3000AA1BBB1B51E107C0AA1FBB1FA617B707B1
:105D400010F0A61BB70B881F991F5A95A9F78095CD
:105D50009095BC01CD0108958F929F92AF92BF9212
:105D6000CF92DF92EF92FF92CF93DF93EC016881A5
:105D700079818A819B81611571058105910521F4E5
:105D800064E279ED8BE597E02DE133EF41E050E0FF
:105D90000E943C2E49015A019B01AC01A7EAB1E4E3
:105DA0000E94E32D6B017C01ACEEB4EFA5019401E0
:105DB0000E94F12DC60ED71EE81EF91EF7FE06C082
:105DC00081E0C81AD108E10880E8F80AC882D982BF
:105DD000EA82FB82C701B6019F77DF91CF91FF90E6
:105DE000EF90DF90CF90BF90AF909F908F900895ED
:105DF0000E94AC2E089586E091E00E94AC2E08959A
:105E00006093060170930701809308019093090144
:105E100008952F923F925F926F927F928F929F92FE
:105E2000AF92BF92CF92DF92EF92FF920F931F93A8
:105E3000CF93DF938B01EA016115710521F0DB013E
:105E40008C9311969C93209739F09E012250310932
:105E50002332310508F0D8C07C016701BFEFCB1AAF
:105E6000DB0A5601F7016080862D90E00E943B30EE
:105E7000892B11F07601F1CFFDE26F120AC05701B4
:105E800082E0A80EB11CD70111966C907724739410
:105E90000BC0BBE26B1207C05701E2E0AE0EB11CB3
:105EA000D70111966C90712CCE018F7E892B89F4CD
:105EB000B0E36B1237C0F50180818F7D8835D1F456
:105EC0006180F2E0AF0EB11C872D8260782EC0E1B8
:105ED000D0E0CA30D10551F1C031D10521F0C83030
:105EE000D10599F409C0CC24CA94DC2CEC2CAFE089
:105EF000FA2E22C0209769F7C8E0D0E0CC24CA94DB
:105F0000DC2CEC2CFFE1FF2E17C06FEF7FEFCB01F5
:105F10009E01442737FD4095542F0E941A2E690197
:105F20007A010AC02097A9F6CAE0D0E0E9E9CE2EAE
:105F3000DC2CEC2CE9E1FE2EF50160E020E030E005
:105F4000A9014E01AA2497FCA094BA2C1F0170ED60
:105F5000572E560CA9E0A51570F48FEB860D8A31EB
:105F600018F499EC592E06C08FE9860D8A3148F550
:105F700089EA582E560C852D90E08C179D070CF55C
:105F80006F3FD9F0C216D306E406F50698F0C501B6
:105F9000B4010E94F62D9B01AC01852D90E0A0E09C
:105FA000B0E0280F391F4A1F5B1F281739074A071F
:105FB0005B0710F46FEF01C061E03196D1016C9086
:105FC000C5CF0115110551F0662311F0319703C0BB
:105FD00071FE04C03297D801ED93FC9370FE07C0A8
:105FE00050954095309521953F4F4F4F5F4F67FF3C
:105FF00010C082E290E090938D0680938C066FEF44
:106000007FEF8FEF9FEF07C060E070E080E090E0EF
:1060100002C0B901CA01DF91CF911F910F91FF908A
:10602000EF90DF90CF90BF90AF909F908F907F9038
:106030006F905F903F902F900895FC0188279927DB
:10604000E89421912032E9F3293010F02E30C8F382
:106050002B3241F02D3239F4689404C00E946F3025
:10606000820F911D219120532A30C0F31EF4909588
:1060700081959F4F0895911150C0803219F0895039
:106080008550D0F7089548EC53E00E9448300895B9
:10609000FA01A191B081009719F41097E1F0CD01B8
:1060A000DC01CD010D90002011F4C00113C0FB01F3
:1060B0002191222319F02015D9F7F3CFFB0121916B
:1060C000201519F41E92119606C02223C1F70D90D7
:1060D0000020A1F7D001FA01A193B08308957AE0DE
:1060E000979F902D879F802D910D11240895F999E8
:1060F000FECF92BD81BDF89A992780B50895262FCD
:10610000F999FECF1FBA92BD81BD20BD0FB6F8949C
:10611000FA9AF99A0FBE019608959927882708954B
:04612000F894FFCF21
:1061240000008E06200001000000FF0002000200B3
:10613400020002000200020002000200020002004B
:106144000200020002000200020002802500000595
:10615400400AA1204EA50020244EA52C2330C012B5
:1061640000001A400AA1204EA5001B1E27522C2312
:10617400308025000005400AA1204EA50020244EB1
:10618400A52C2330004B000006400AD0009D490096
:106194007B289D492C233000E1000005400A45017D
:1061A400D7DC03B81E0EBF00232E48E801008A4046
:1061B4000A6001555502AD1E20000023C801545841
:1061C4002074696D656F75742100596573004E6F95
:1061D400002C00386368004E2F41002C205B005DCA
:1061E4002028002900486F70206368616E6E656C1A
:1061F400200020402000456E746572696E6720613E
:1062040064617074697665206368616E6E656C2084
:1062140073656C656374696F6E2C207069636B6958
:106224006E673A007363616E6E6572206D6F6465AC
:10623400004E4F5420454E41424C45440053656E38
:1062440064696E672073657474696E677320746F14
:106254002052580A00526573657474696E6720731E
:10626400657474696E6773206F6E2052580A00411A
:10627400626F727465642065646974730A00696E80
:1062840076616C69642073656C656374696F6E0014
:106294000D0A496E76616C696420696E70757420AC
:1062A4002D2064697363617264656421070053651A
:1062B4007474696E677320736176656420746F20EB
:1062C400454550524F4D0A005265766572746564B7
:1062D4002073657474696E67732066726F6D2045F0
:1062E4004550524F4D0A004C6F61646564206661ED
:1062F40063746F72792064656661756C74730A00E7
:106304004B657920616E64206368616E6E656C73A1
:106314002072616E646F6D697A65640A004F7065FE
:106324006E4C52536E6720545820737461727469B2
:106334006E672000206F6E20485720006D6F6475D3
:106344006C65206C6F636B65643F00342B340038DC
:1063540000382B340031320031322B340031360016
:1063640050504D0052535349005344410053434C41
:1063740000525844005458440041494E004C424590
:1063840045500053504B54524D0053425553005303
:10639400554D44004C4C494E440000070B0C101161
:1063A4001500B7012B032F033103350338033D03D5
:1063B400B7014003440349034D03510355035903F3
:1063C4005D0363036A036F0374038D028D028D0200
:1063D4008D02160A13223129000000001C2C212AE8
:0863E400C22BEF2BD42B112C6E
:107E00000F92CDB7DEB7112484B714BE81FFF1D035
:107E100082E08093C00088E18093C10086E0809377
:107E2000C20080E18093C4008EE0CDD088249924E4
:107E3000CC24C394F5E0DF2EE1E1EE2E73E0F72EC3
:107E4000B6D0082F813479F4B2D08983C2D0898129
:107E5000823811F481E005C0813811F485E001C059
:107E600083E09ED09AC0823411F484E103C085344B
:107E700019F485E0B6D091C0853561F498D0082F0B
:107E800010E095D090E0982E8824802A912A880CC2
:107E9000991C82C0863521F484E0A3D080E0E1CF34
:107EA000843609F04CC083D082D0A82E80D0B82E62
:107EB00000E011E07CD0F80181938F01AE16D1F77C
:107EC00088D0FB2DF53489F4E0E0F1E00BC0F9999E
:107ED000FECF92BC81BC0894811C911C819180BD15
:107EE000FA9AF99AEA1598F358C08B2D863409F05E
:107EF00054C0F401F7BEE89507B600FCFDCFF401CD
:107F0000A0E0B1E02C9130E011968C91119790E0B7
:107F1000982F8827822B932B12960C01C7BEE895C9
:107F20001124329681E0A038B80761F7F401D7BE7A
:107F3000E89507B600FCFDCFE7BEE8952EC0843774
:107F4000F1F435D034D0182F32D0B82E42D0FB2DDA
:107F5000F63421F4F40105914F010CC0FB2DF534EA
:107F600049F4F999FECF92BC81BC0894811C911C04
:107F7000F89A00B5802F14D0115049F70EC08537FC
:107F800039F427D08EE10CD085E90AD08FE069CF93
:107F9000813511F488E017D01CD080E101D050CF9A
:107FA0009091C00095FFFCCF8093C600089580910A
:107FB000C00087FFFCCF8091C00084FD01C0A89560
:107FC0008091C6000895E0E6F0E098E19083808318
:107FD0000895EDDF803219F088E0F5DFFFCF84E10E
:107FE000DFCF1F93182FE3DF1150E9F7F2DF1F9166
:0E7FF0000895282E80E0E7DFEE27FF27099492
:027FFE0001057B
:0400000300007E007B
:00000001FF
